:020000001628C0
:080008001628202091000439A4
:10001000031D7B209118452011183C2000008316F9
:1000200008308100831281016300052883161F3088
:100030008500F03086008312FF3086008B1505287E
:100040000608C039910033200608C0399100910C90
:10005000910C910C910C910C910C110882070434B5
:1000600001340234003414308E008F018E0B392895
:1000700008008F0B392835280F30860006101930FC
:10008000900085204E20732008000F3086008610D7
:100090003730900085204E20732008001108013968
:1000A000031D53286328023092000614013090008B
:1000B00085200610013090008520920B55280130D4
:1000C00090008520080002309200861401309000D4
:1000D00085208610013090008520920B6528013024
:1000E00090008520080006110F309000852006152D
:1000F0000F308600080006110610861001309000AF
:10010000852006150614861408008920900B852882
:100110000800831607308100831281010E308F00A2
:100120008E00811A9428912881018F0B91288E0BC3
:040130009728080004
:02400E00F13F80
:00000001FF
